:100000006FC0B9C187C086C085C084C083C082C0AC
:1000100081C080C07FC07EC07DC07CC07BC07AC0F4
:1000200079C078C077C016032800530029004E001D
:10003000450053005F0075007300620018037200F2
:100040006100700068006E00650074002E006E0094
:100050006500740004030904090222000101008004
:100060003209040000010300000009210101000120
:100070002200000705810308000A120101010000A7
:1000800000088117960A0001010200010501090517
:10009000A1010901A10009300931150025037504EA
:1000A00095028102C005091901290815002501756D
:1000B0000195088102C005010905A1010901A100FE
:1000C0000930093115002503750495028102C00528
:1000D000091901290415002501750195048102C043
:1000E00011241FBECFE5D4E0DEBFCDBF10E0A0E6F7
:1000F000B0E0E6E8FBE002C005900D92A238B1073F
:10010000D9F710E0A2E8B0E001C01D92A93CB10708
:10011000E1F753C375CFCF93DC01C62F693008F0E8
:10012000C8E02BE490919A0090FD23EC809162004E
:1001300087FF04C09F5F90939A0003C08FEF809366
:1001400062002093B300E4EBF0E02C2F21502F3F0E
:1001500019F08D918193FACF6C2F84EB90E0BDD292
:10016000CC5FC0936200CF9108951F93CF9390917D
:10017000C300992309F483C0935097FD7EC0E2E841
:10018000F0E0E091B200EF5F40E0C0E88091C00095
:100190008D3209F06EC0983009F06BC08081807696
:1001A00009F064C02FEA30E04093AF0081818823DA
:1001B00021F44093B00042E04EC0853021F48281AA
:1001C0008093C40048C0863091F5C0EC83818130B3
:1001D00021F442E12AE730E03EC0823021F442E2DD
:1001E00028E530E038C0833099F48281882321F4F7
:1001F00044E024E530E02FC0813021F448E12CE3D5
:1002000030E029C0823039F546E126E230E023C0F3
:10021000813221F449E02AE630E01DC08232D9F46F
:100220004091B1002091C7003091C80014C08830BF
:1002300021F441E026EC30E00EC0893021F48281C7
:100240008093C60008C08A3011F441E004C08B30AE
:1002500011F440939A003093C2002093C10087812B
:10026000882339F48681841720F402C0CF0139D263
:10027000482FC0939800409364001092C30090915F
:1002800064009F3F09F44FC08091630087FF4BC01B
:10029000692F993008F068E0961B909364001BE486
:1002A0008091980080FD13EC8F5F80939800A7EAFF
:1002B000B0E0E091C100F091C200962F915086FF0E
:1002C00013C09F3FB9F084919D012F5F3F4FAF0155
:1002D0004F5F5F4F9150E157F04011F48091B100B2
:1002E0008C93D901FA01EDCF9F3F21F081918D933D
:1002F0009150FACFF093C200E093C1007727C62F48
:10030000693040F487EA90E0E8D19C2F9C5FC830C8
:1003100030F402C01EE192E08FEF809364001093EE
:10032000A6009093630080B3857019F01092990035
:1003300011C080919900882369F494E680B3857098
:1003400049F49150D9F781E0809399009093C400CB
:100350009093BF00CF911F91089582E890E0809321
:10036000BE000B968093B20085B7836085BF8BB7C4
:1003700080648BBF08950F930FB70F93809BFECFC0
:10038000809B06C0809B04C0809B02C0000000C010
:100390001F933F932F9331E014E000B3102710FD1B
:1003A00032E0102F3A95C9F700FDE7C000B31027DF
:1003B00017952FE72795DF9310B30127079527950A
:1003C000CF93C091BE0000B31027179527953BE04F
:1003D000D0E04F9310B30127079527954FEF00000A
:1003E00055C0809BFECF809B06C0809B04C0809B35
:1003F00002C0000000C0DF9100C0CDCF10B3157067
:1004000079F1407C2C6F13C000B3057049F141783D
:100410002C6F15C0057021F1102F2C6F00B319C07F
:1004200000B30570E9F04E7F2C6F18C038F300B3AD
:100430000570B1F0102717952795243028F310B3D5
:10044000012707952795422749934FEF00B32430A2
:1004500008F3102717952795243010F310B3157063
:10046000E1F10127079527952430F0F000B30570DE
:10047000A1F11027179527952430E0F010B301273C
:10048000079527953A9541F12430D0F000B30570D7
:1004900021F11027179527952430C0F010B30127BC
:1004A000079527952430C2CF10B31570B1F04C7F5B
:1004B0002C6FDCCF00B3057081F0487F2C6FDECF4E
:1004C00010B3157051F0407F2C6FE0CF00B3057072
:1004D00021F0407E2C6FE2CF3DC03C2FC091BE008A
:1004E0003C1B00E433300ABFA8F108811981412F79
:1004F0001F772091BF000D3289F1013E79F1093655
:10050000C1F00777033431F51091C500112311F1C3
:100510000091C3000030D1F53430DAF13093C300DC
:100520001093C0000091B200C093B2000093BE00CF
:1005300030C0121779F447FD3AC0309163003F3F55
:1005400029F10FEF00936300C6EAD0E025C0002731
:100550000093C5004F91CF91DF910FC01217B9F7EB
:100560000093C5000FEF00936400009363004F9168
:10057000CF910AB706FD35CFDF9100E40ABF2F9176
:100580003F911F910F910FBF0F911895C0E6D0E0DA
:1005900002C0C1E6D0E032E05F9302B30A7F01609F
:1005A00002BB55E011B3156011BB20E819C03091B2
:1005B00062003F3F59F30FEF00936200C3EBD0E0BE
:1005C000EBCF052710E002BB10C0052710E0089410
:1005D00002BB13C0052710E015C0052710E019C0A5
:1005E00020FF052702BB279517951C3F50F720FFDA
:1005F0000527279502BB17951C3F38F720FF0527D5
:100600002795179502BB1C3F28F720FF0527279544
:1006100017951C3F02BB08F700C0499120FF052732
:1006200002BB279517951C3F80F520FF05272795CE
:1006300002BB17951C3F68F520FF052727951795E6
:1006400002BB1C3F58F520FF0527279517951C3F37
:1006500002BB38F5242F3A9519F60A7F5F9102BB49
:1006600032E03A95F1F71091C400C256D04011F033
:100670001093BF00016011B31A7F02BB0A7F4F9134
:10068000CF9111BB02BBDF9178CF052710E002BBF1
:10069000CACF052710E0089402BBCDCF052710E094
:1006A000CFCF052710E0D3CFA82FB92F8FEF9FEF23
:1006B00041E050EA615070F02D9138E0722F7827B8
:1006C00096958795269570FF02C0842795273A95C1
:1006D000A9F7F0CF809590950895E6DF8D939D93CF
:1006E0000895FC012DE930E03093C2002093C10051
:1006F0008081992780769070809719F5818181306B
:1007000081F4E0919B00F0919C000484F585E02D3C
:10071000C9010995E0919B00F0919C008081992787
:100720000895823049F48FE990E09093C20080935D
:10073000C10081E090E008958A3019F483818093AC
:100740009F0080E090E00895EF92FF920F931F9337
:10075000CF93DF93959AAC01415050408FEF4F3FBC
:10076000580721F180E3E82E85E7F82E012D112DA1
:10077000959823E130E0C7010197F1F7215030400F
:1007800037FFF9CF959AA0E3B5E7C0E0D0E021E3C9
:1007900030E0CD010197F1F72150304037FFF9CF1C
:1007A000415050408FEF4F3F580711F7DF91CF91E5
:1007B0001F910F91FF90EF900895CFE5D4E0DEBF39
:1007C000CDBFC0E001E01C2F8D9AB89A87B3897F16
:1007D00087BB88B3866088BBC09880E395E70197A4
:1007E000F1F786B3992786709070002E02C0959518
:1007F00087950A94E2F78230910531F0039761F012
:1008000081E090E0A1DFFCCFA4D190939C00809385
:100810009B0081E090E007C018D190939C008093EA
:100820009B0082E090E090DFE0919B00F0919C00C3
:10083000848195819093C8008093C70082818093C2
:10084000B1009FEF95BB14BA8AEF82BB87E081BBF2
:1008500080E08150F1F79150D9F782E081BB85E0CB
:1008600083BF0680F781E02D099577DD7894A89500
:100870007CDC002349F0E0919B00F0919C00008417
:10088000F185E02D099500E008B600FE14C091E066
:1008900098BF80919F00882331F0153010F01550DB
:1008A00002C0182FC92FE0919B00F0919C0000849A
:1008B000F185E02D0995E0919B00F0919C00028468
:1008C000F385E02D0995882311F0C1E002C0CC2307
:1008D00071F2809162008F3F51F6C0E0E0919B0081
:1008E000F0919C000484F585E02D8DE990E0099558
:1008F000E0919B00F0919C0060818DE990E00BDC21
:10090000B6CFA49AA59AA398AB9AAD9A95B39095B1
:1009100085B3892385BB089590E0AC9A80E38A95DE
:10092000F1F7AC9828E130E040E050E067E070E09B
:10093000822F8A95F1F7AD98990F9B9B9160822F3A
:100940008A95F1F7AD9A6150704077FFF1CF90939F
:10095000A00028E130E040E050E067E070E0822F46
:100960008A95F1F7AD9896959B9B9068822F8A9512
:10097000F1F7AD9A6150704077FFF1CF9093A100ED
:10098000089542E050E062EA70E080EA90E0EED044
:10099000992787FD90950895CF93DC01892B09F461
:1009A0004AC08091A000C091A100E1E0F0E0BF0149
:1009B000482F552740FF02C0E2E0F0E041FF02C0AF
:1009C000E0E0F0E042FF02C062E070E043FF02C0FE
:1009D00060E070E084E0660F771F8A95E1F78E2F64
:1009E000862B8C939A01220F232F221F330B3195D4
:1009F000CA0180749070E5E095958795EA95E1F7D6
:100A0000282BCA018072907073E0959587957A952E
:100A1000E1F7282B4071507055954795242B8C2F6A
:100A200099278F70907034E0880F991F3A95E1F7FD
:100A3000282BFD0121838091A0009091A10090932B
:100A4000A3008093A200CF9108958CE890E08638AF
:100A5000910509F0959890936A008093690085E666
:100A600090E00895A49AA59AA398AB9AAD9A95B3ED
:100A7000909585B3892385BB089590E0AC9A80E377
:100A80008A95F1F7AC9828E130E040E050E067E06B
:100A900070E0822F8A95F1F7AD98990F9B9B91603A
:100AA000822F8A95F1F7AD9A6150704077FFF1CFB0
:100AB0009093A40008958091A4009091A500891BB3
:100AC000992787FD90950895FC01892BE9F161E054
:100AD00070E09B018091A400482F552740FF02C081
:100AE00062E070E041FF02C060E070E042FF02C0DF
:100AF00022E030E043FF02C020E030E0A4E0220F1B
:100B0000331FAA95E1F7862F822B80839A01220F4B
:100B1000232F221F330B3195CA018074907065E03A
:100B2000959587956A95E1F7282BCA018072907098
:100B300033E0959587953A95E1F7282B40715070F1
:100B400055954795242B21838091A4008093A5007F
:100B5000089586EB90E08638910509F0959890937A
:100B600078008093770083E790E00895FB01DC0133
:100B700004C08D910190801921F441505040C8F774
:060B8000881B990B08958B
:100B86005AD2FFFFFF02002A00000081048C04C134
:100B960004CC0402002A00000032053D055B056412
:020BA600050048
:00000001FF
